:020000040000FA
:10000000831628308100103085000F30860083125F
:100010008501A301BF20A30A2308063A0319122869
:1000200038200B2834200B28A100A2012C20A10D80
:10003000031821282320A20A2208240603190800F5
:10004000172829201B280630850031208501312002
:100050000800063085003120312031208501312013
:100060000800A00B312808002B202C20A301080039
:1000700006080F390F3AA400820747284D28532855
:100080005D285F2874288928A328A828B428010897
:100090000139A400A40AB720142881194728033085
:1000A000A400B720142801080339A400A40A0430CE
:1000B000240603195F28B7201428B7201428B72076
:1000C0000F39632014288207003410342034403460
:1000D0006034703480349034A034B034C034D034C0
:1000E0000034103420344034B7200F3978201428DD
:1000F0008207F834783438341834083400348034C3
:10010000C034E034F034F8347834383418340834F7
:100110000034B7200F399220A10003398207152837
:10012000A403152882075434CC3478343034E034B6
:10013000B434843448341434B1348934413491347F
:10014000A93451341134811953280530A40074287E
:10015000B7200339AF20A1000739A4001528820772
:100160006D342534E434343481195328A828A60A80
:100170002618BD280108A5000800250E0800C62085
:100180003420C6203420C62034200800CA20CA20CB
:0E019000CA2008000430A4001030142008001B
:02400E00F33F7E
:00000001FF
